:1000000019C020C01FC01EC01DC01CC01BC01AC00C
:1000100019C018C017C016C015C014C013C012C034
:1000200011C010C00FC00EC00DC00CC00BC00AC064
:1000300009C008C011241FBECFEFD2E0DEBFCDBF84
:100040000AD13BC1DDCF85B38823E9F385BB429A52
:10005000242D47FE02C038980AC0822D20FE04C01D
:100060004EEF242E282202C081E086B9389A952DC1
:1000700057FE02C039980AC0822D21FE04C03DEF10
:10008000232E282202C082E086B9399A422E440CDF
:10009000592E550C42980895439A85B38823E9F365
:1000A00085BB3898399843988FE295B39923E9F343
:1000B00095BB8150D1F7089522242394439A442478
:1000C0008FEC582EC0DF4398BEDF22242394BBDF81
:1000D000BADFB9DFB8DFB7DFB6DFBFEC5B2EB3DF67
:1000E000B2DFB1DFB0DFAFDFAEDFA0E84A2EABDFBB
:1000F000AADFFFEC5F2EA7DFA6DFA5DFA4DFA3DF6B
:10010000A2DFA1DFA0DFEFEC5E2E9DDF9CDF9BDF97
:100110009ADF99DF98DF97DF96DF7FEC572E93DF2A
:1001200092DF91DF90DF8FDF8EDF8DDF8CDF6FEC72
:10013000562E89DF88DF87DF86DF85DF84DF83DF78
:10014000442488B1822580FF02C050E8452E7BCF31
:1001500022242394439A4424532C75DF4398532C30
:1001600072DFB3E02B2E482C55246DDF6CDF82E06C
:10017000282A5A2C68DF67DF66DF65DF64DF63DF0C
:10018000432C61DF330C5FDFA0EA4A2E552488B18F
:10019000822581FF02C0F0E85F2E55DF532C53DF2C
:1001A000532C51DF4C2C55244EDF4DDF5E2C4BDFA2
:1001B0004ADF49DF48DF47DF46DF432C44DF330CAB
:1001C00042DF4424552488B1822581FF02C0E0E843
:1001D0005E2E39DF892D9927482E532C34DF532C7E
:1001E00032DF8B2D9927582E2EDF2DDF2CDF2BDFD2
:1001F0002ADF29DF432C27DF330C25DF4424552455
:1002000088B1822581FF02C050E8552E1CDF8D2D5C
:100210009927482E532C17DF532C15DF8F2D992744
:10022000582E11DF10DF0FDF0EDF0DDF0CDF432C48
:100230000ADF330C08DF442488B1922D822580FF29
:1002400002C020E8422E552488B1892781FF02C0D0
:1002500090E8592EF8CE0F931F93CF93DF9380E150
:1002600085BF8CE787BD8EE388BD82E084BD81E0D9
:1002700085BD8CE087B988248A94982CAA24AA94F6
:10028000BA2CCC24CA94DC2CEE24EA94FE2C02E096
:1002900011E006B916B9C0E4DFE1FEDE2197E9F707
:1002A000C0E4DFE109DF2197E9F7C0E4DCE93324AA
:0E02B0003A944EDF2197D9F7ECCFF894FFCFA8
:00000001FF
